:020000040000FA
:020000000528D1
:0800080005288501860107307F
:100010009F008316A730810012308500860183126D
:100020008501851811281430422085181128051AD9
:10003000172886010430A4002B20A30003191028E0
:100040002B202302031D1028A40B20282308860040
:10005000851C28281028810134200108A500203C97
:10006000031CA501250808003230A000A00B36288B
:1000700008000430A0005130A100A10B3D28A00BC6
:0E0080003B280800A2003920A20B43280800EC
:02400E00103F61
:00000001FF
